:020000040800F2
:1000000070050020D90000085D1E0008991C00083A
:1000100000000000000000000000000000000000E0
:10002000000000000000000000000000A71E000803
:100030000000000000000000A51E0008A91E000826
:10004000EB000008EB000008EB000008EB000008E4
:10005000EB000008EB000008EB000008EB000008D4
:1000600000000000EB000008EB000008EB000008B7
:10007000EB000008EB00000800000000EB000008A7
:1000800000000000EB00000800000000000000007D
:10009000EB00000800000000EB000008EB00000887
:1000A000EB000008EB000008EB000008B523000897
:1000B000EB000008EB00000800000000000000005A
:1000C0000448854600F04CFB00480047252D0008F9
:1000D000C046C046700500200448804704480047D9
:1000E000FEE7FEE7FEE7FEE7FEE7FEE71D1F00086E
:1000F000C100000830B50B46014600202022012433
:1001000009E00D46D5409D4205D31D469540491B4B
:100110002546954040191546521E002DF1DC30BD94
:10012000F0B51FB40646002082B005464024019178
:1001300000901BE0019922460F46304600F0F5F88A
:10014000049A059B801A994110D3104619462246FD
:1001500000F0DBF8361A8F4101972246012000217A
:10016000009F00F0D2F838184D4100902046641EE0
:100170000028DFDC019B00982946324607B0F0BD1D
:10018000D2B201E00270401C491EFBD2704700222F
:10019000F6E710B513460A4604461946FFF7F0FF86
:1001A000204610BD024670B54A40D30FDB07400021
:1001B0002DD04A002AD0010E140E00021202091995
:1001C000400A520A8418E50104465443000A120A00
:1001D0002E045043A4194219200CC543AA18120C2E
:1001E0000125AD03521C521912047F39240400D09A
:1001F000521C104301D44000491EC2B20C06C00973
:100200002018401C4008802A02D003E0002070BD66
:1002100040084000002900DA0020184370BD70B586
:1002200002464A40D50F40004A00ED0740085208F8
:10023000002814D0002A12D0C40DD30D4102012091
:10024000C0055202490A520AE41A091812187D34EC
:10025000914201D3641C00E04900002C01DA002027
:1002600070BD0023914201D3891A0343400849001D
:100270000028F7D100290AD0914202D10121C907F3
:1002800005E0914201D2012101E00121C943E005CD
:10029000C018401900F05AF870BDC217C10F504085
:1002A00010B54018CA079623002100F057F810BD7A
:1002B000C20F410040020123400ADB05D207090EAC
:1002C000C0187F2901DA00207047962903DC9623A5
:1002D000591AC84001E096398840002AF4D04042BB
:1002E0007047C20FD207400040080BD0C10D072352
:1002F000DB01C91840020905400A1143C208400742
:100300001143704700200146704710B5202A04DBD6
:100310000146203A9140002010BD914020239C1AB4
:100320000346E3401943904010BD10B5202A04DB7A
:100330000846203AD040002110BD0B46D340D040A3
:100340002024A21A91400843194610BD002904DA5E
:10035000401C490001D140084000704770B400249F
:10036000050C05D11024000402D1002921D011244C
:10037000050E01D100020834050F01D10001241D32
:10038000850F01D18000A41C002801DB4000641C03
:10039000002908D020252E1B0D46F540A14000D095
:1003A00001212943084301061B1B000ADB1D02D55E
:1003B000002070BC7047DB05181880180029F8DA97
:1003C000401C4900F5D170BC400840007047000057
:1003D000F0B507460846584087B0C00F0490480063
:1003E0000E46590040084908BC1A884105D23846D3
:1003F00031461E4617460B46024658004008104339
:100400004DD0300D039040055900400D490D059029
:10041000401A0290402873DA18030121000B0905E5
:100420000843019004980092002806D01146019AD2
:1004300049420020904100910190029840210A1AFF
:1004400001990098FFF761FF05460C466B4607CB04
:1004500000F098F9C0197141039A0E0D0023D717C7
:1004600056401A467A40164344D0049A002A2DD0AA
:10047000029A012A039A15DC1205C01A914101263D
:100480003605001C7141D20F059ED20700930192E0
:1004900002962A46234600F095F907B0F0BD38468B
:1004A0003146FAE71605234A0F46B218C01AB7417B
:1004B00001210905001C4F4100187F411146181801
:1004C0007941E20F10436D19644113E0E2076D08B2
:1004D00015436408C2071443039A01261205C01A83
:1004E00091413605001C7141CE0740083043490850
:1004F000C01851412A46234600F057F9CDE7FFE7DF
:10050000049801224000C117121A00238B4104985D
:100510003146C417381AA141EEE730B40124E4078C
:10052000634030BC54E730B40124E407614030BC80
:100530004EE700000000E0FFF0B51FB488B00B9953
:100540000998002448400999C00F490049080991B9
:10055000C0070B990090490049080B910999089828
:10056000A64608431CD00B990A98084318D009984E
:1005700001244000420D4800410D09982405000364
:10058000000B204309900B980003000B20430B90B5
:1005900050181C494018002201901446104605E0EE
:1005A000002001460DB0F0BD032801DA034600E04B
:1005B00003239C46C11A0AAE0AE05F0008ADED5B5A
:1005C0004F00F75B7D430027AA187C41491C5B1E46
:1005D0006145F2DD410004AB5A522104120C0A437A
:1005E000240C401C0828DFDB01980290009970461B
:1005F00001910090059B049A0799069800F0E2F893
:10060000D0E700000DFCFFFFF0B50C465C4085B064
:10061000E40FE40703944C00002664085900944654
:10062000490802460296224321D062460A431ED060
:100630006200570D4A000E032303550D01240246A4
:100640002C492405781B1B0B360B401823432643EB
:10065000614600901C46501AB44103D30098401CD8
:10066000009002E0921800985B41002803DA002015
:10067000014605B0F0BD0020012109050746864668
:1006800011E064461D46141BB54106D36546521B56
:10069000B341744607430C43A646CD0740084908BA
:1006A000284392185B4105460D43EAD11046184392
:1006B00013D06046194650407140084306D060464A
:1006C000101AB34106D20122002306E000220123C2
:1006D000DB0702E00122D243531000987446010563
:1006E000381C6141029C039D0019694100F05DF8CE
:1006F000BFE70000FD0300004A0009030123090BC6
:100700001B0519430A4B10B5520D9A4202DA00201C
:10071000014610BD064B34339A4203DC9A1AFFF7A8
:1007200004FE10BD034BD218FFF7EFFD10BD000013
:10073000FF030000CDFBFFFF10B5002904DB0124FF
:10074000E40740428C412146002B04DB1C46012378
:10075000DB075242A341994200D1904210BD0000F4
:10076000064C0125064E05E0E36807CC2B430C3C04
:1007700098471034B442F7D3FFF7A6FCF42D0008D5
:10078000142E000810B5202A06DBCB170846203AA5
:100790001041C1170B4306E00B461341D040202403
:1007A000A21A91400843194610BD10B5002B08DA73
:1007B0000024401C614192185B411A4301D140085A
:1007C000400010BDF0B51FB482B005460C0003D048
:1007D000084601F007FE02E001F004FE2030024668
:1007E000009021462846FFF790FD049B059A044699
:1007F0000F4618431143084314D0184610431BD02A
:10080000009840210A1A18460599FFF78EFD054603
:100810000E46009A05990498FFF777FD084305D026
:10082000012004E02046394607B0F0BD0020C11782
:1008300005430E432C43374300990E986305401A35
:100840007905E40A00220C43FD0A0A3002D5002093
:100850000146E9E70105101969410C9C0D9D00193D
:100860006941FFF7A2FFDFE738B5044606480549AE
:100870000068FFF73FFC604300E0401E0090002846
:10088000FBD138BD40420F000400002070B50024A9
:1008900005252D0704E0641CE4B2012002F02EFAC5
:1008A0001021284600F020FB002802D0C82CF2D3EB
:1008B00010E0C82C0ED2002404E0641CE4B2012035
:1008C00002F01CFA1021284600F00EFB002803D08D
:1008D000F02C04D3012070BDF02CEED3FAE70020F9
:1008E00070BD000070B500F07DF800F065F8FFF70E
:1008F000CDFFCC2000F082F8BE2000F07FF800F0A1
:100900004CF8044600F049F8072805D9C043E143F4
:10091000C0B2CCB2002500E001250002001900B2EF
:10092000FFF7BBFC0549FFF73DFCFFF7C1FC00B238
:10093000002D01D1404200B270BD00000000203FF8
:1009400010B5052001221021000700F0D2FA00F0B6
:1009500033F8FFF79BFF10BD10B5052424070022D4
:100960001021204600F0C5FA022002F0C7F901224A
:100970001021204600F0BDFA0C2002F0BFF9102132
:10098000204600F0B1FA002801D0012200E0002248
:10099000322002F0B3F9104610BD70B500250124D5
:1009A000FFF7DAFFC00169080843641CE4B2C5B26E
:1009B000082CF5D9284670BD10B50524240700225F
:1009C0001021204600F095FA054802F097F901221F
:1009D0001021204600F08DFA0F2002F08FF910BD93
:1009E000EE02000010B5FFF7E7FFFFF74FFFCC2046
:1009F00000F004F8442000F001F810BD70B50124A7
:100A0000052605463607E807C00F6D0800280ED0FA
:100A100000221021304600F06CFA022002F06EF93C
:100A200001221021304600F064FA3C200DE0002243
:100A30001021304600F05DFA3C2002F05FF90122FF
:100A40001021304600F055FA022002F057F9641CDC
:100A5000E4B2082CD7D970BD70470000F8B506463F
:100A60000D464036317C01290DD0012131740168D9
:100A70008A68520709D5416D202211434165002043
:100A800030740120F8BD0220F8BD174B6A68D80504
:100A900047109A42154C8A6A2B6812D05B035B0B95
:100AA0001A438A622968490305D5A1680143A160F8
:100AB0000A20FFF7D9FE2868800312D5A0683843C2
:100AC0000EE05B035B0B9A438A622968490302D5F7
:100AD000A1688143A1602868800302D5A068B8435B
:100AE000A06000203074F8BD011000000027014014
:100AF00070B5040006D0606D2646002540360028FB
:100B000002D006E0012070BDA5653574204600F0D6
:100B1000D3F8606DC00603D421688868400705D506
:100B2000606D1021084360653574EBE7606DFF224E
:100B30000132904302221043606588688207920F59
:100B40005B48012A02D10A68D2072BD103236268CD
:100B50009B079A4205D05B429A4202D05B009A42C0
:100B600009D10A69920092080A6121680A696368DA
:100B70001A430A610CE00A69920092080A618168CE
:100B80000F22920491438160816862681143816001
:100B90002168CA6818239A43CA602168CA68A36892
:100BA0001A43CA60816801225206914381608168BC
:100BB000A28E52061143816020688168C90004D466
:100BC000816801221207114381602068C168394A97
:100BD0001140C1602069E168022825D0002001434E
:100BE000204620300278037B52035B001A431143F6
:100BF000226B1143A26992031143E269D2031143AC
:100C00002268D3681943D160616A0A46FF3AC23A42
:100C100005D0A26A11432268D3681943D160427893
:100C20000121012A02D00BE00420D8E70078002837
:100C300023D0606D202210436065A06D0843A0653D
:100C4000E06B012820681FD00169C90703D0016942
:100C500049084900016120684169C908C90041612A
:100C600020684169A26B11434161A565606D8008F0
:100C70008000401C6065002070BD2068C2680123B0
:100C80001B041A43C260DBE70269FF239B009A43FF
:100C9000026120680269236CA66C1A43636C3343BB
:100CA0001A430261206802690A430261D3E7000027
:100CB000002701401902FEFF10B586B0044614213A
:100CC0006846FFF764FA0E492068884216D10D483D
:100CD000416B421511434163C16A01221143C16254
:100CE000C06A6946104005902020009003200190C2
:100CF000002002900520000700F03AF806B010BD71
:100D0000002401400010024070B50024014620314B
:100D10004A79022A03D00421C163012418E0026841
:100D200013680E25AB431360026813685B085B0011
:100D30001360436C1C221340012215469D40036C36
:100D40005D604A7100220A71816B002900D08847DA
:100D5000204670BD70B5044600F0D2F80546601C10
:100D600000D0641C00F0CCF8401BA042FAD370BD48
:100D7000F8B500230124A2E027469F403A4070D0F6
:100D80004D68022D01D0122D14D1DD08AD002D18B3
:100D900000952D6A5E07AC46F50E0F26AE46AE40B6
:100DA0006546B543AC460E697546AE4065462E4372
:100DB000009D2E624D68012D05D0022D03D0112D0E
:100DC00001D0122D16D185680326AC465D00AE46D3
:100DD000AE406546B543AC46CE687546AE40654606
:100DE0002E43866046680D79BE43ED06ED0F9D40AB
:100DF0003543456006685F000325BD40AE46AE43FF
:100E00000D79B446AE07B60FBE4065462E43066068
:100E1000C6687546AE438D68BD403543C5604D68B4
:100E2000ED004BD5294D6E6B26436E639E08284D11
:100E3000B6007519AC46AD689E07360F0F27B74050
:100E4000BD4305273F07B84201D1002715E0214FD8
:100E5000B84201D1012710E01F4FB84202D102274A
:100E60000BE02BE01D4FB84201D1032705E01C4FDA
:100E7000B84201D1052700E00627B7402F43654659
:100E8000AF60184D2E684F689643FF0300D5164398
:100E90002E606E684F689643BF0300D516436E60A0
:100EA000AE684F689643FF0200D51643AE60EE6809
:100EB0004F689643BF0200D51643EE605B1C0A687C
:100EC0001546DD4000D057E7F8BD00000010024095
:100ED000000001400004005000080050000C0050C9
:100EE000001C0050000401400069084000D00120AF
:100EF0007047002A01D0816170478162704700000D
:100F000001480068704700000000002070B50246EC
:100F100040325378202B1CD11378012B19D0012398
:100F2000137024245470046825689D432560046868
:100F300025681E03B5432560046825680D432560B8
:100F40000068016819430160202050700020107073
:100F500070BD022070BD70B5024640325378202B20
:100F60001BD11378012B18D0012414702423537043
:100F700003681D68A5431D6005682B680F263602AF
:100F8000B3430902194329600068016821430160E5
:100F9000202050700020107070BD022070BD000035
:100FA00070B5040006D02546403568780026002834
:100FB00002D005E0012070BD2E70204600F04AF8F6
:100FC00024206870206801684908490001600F21E9
:100FD0006068090688432168086121688A680120E1
:100FE000C00382438A60E1680129A16808D02122F8
:100FF0009202114322689160E168022902D005E063
:101000000143F7E701212268C902516021684A685B
:101010000F4B1A434A602168CA688243CA606169FB
:1010200020690843A169090208432168C860216A50
:10103000E0690843216808602068016801221143C3
:1010400001606664202068702663AE70002070BD69
:101050000080000210B586B0044614216846FFF7F0
:1010600096F81149206888421BD1104CE16A022091
:101070000143E162E16A0140032005918002009092
:10108000122001900120029003200390062004907A
:1010900069460748FFF76CFEA06B012189050843EC
:1010A000A06306B010BD00000058004000100240D0
:1010B0000004005002480168491C016070470000AC
:1010C0000000002010B508480024016840221143A8
:1010D0000160204600F00AF8002801D0012401E058
:1010E00000F01CF8204610BD0020024070B50546F7
:1010F00009487D210024C9000068FEF7FBFF00F0CD
:10110000F9FB002801D0012404E000222946501EEA
:1011100000F01AF8204670BD040000200448416B1E
:10112000012211434163816B0204114381637047C3
:1011300000100240C106C90E012088400149086024
:101140007047000000E100E010B500F089FE10BD1E
:10115000F8B504460078544D800672D5524E0027EB
:10116000403EB06BC00004D4B06BA9050843B06327
:1011700001274E480168C90511D401688215114341
:101180000160FFF7BDFE009005E0FFF7B9FE009992
:10119000401A642837D845480068C005F5D532683C
:1011A0000321090560680A400140914208D081038B
:1011B000890F032904D13168890301D50120F8BDC5
:1011C0002A69032109040A4022D0084090421FD016
:1011D000207880061CD528692A6988430121C90422
:1011E0000A432A612A698A432A612861C0050FD50A
:1011F000FFF786FE009008E0FFF782FE0099411A93
:101200002B48814201D90320F8BD28698005F3D518
:1012100061688803800F032805D132680005824386
:1012200001400A43326028690322616812041140B8
:1012300008432861002F04D0B16B012000078143CF
:10124000B1632078C00705D0E868A16880088000F5
:101250000843E8602078800705D5E8680C218843BA
:10126000E1680843E8602078400706D5E868032174
:101270008902884321690843E8602078000706D581
:10128000E86803210903884361690843E86020781E
:10129000000606D5E868032189048843A16908434C
:1012A000E8600020F8BD00004010024000700040DF
:1012B00088130000F8B50E4605007DD0534800683D
:1012C000C007C00FB0420AD250480168490849001F
:1012D000314301600068C007C00FB04271D1287867
:1012E0004B4C800705D5E068F0218843A968084386
:1012F000E0602878C00752D06868022817D0032819
:1013000018D02168012818D08905002959DAE16828
:10131000890889000143E160FFF7F2FD696807462B
:10132000022912D003291CD0012926D033E02168DC
:101330008903EAE721688901E7E74907E5E7FFF75D
:10134000DFFDC11B3348814223D8E0680007800FCE
:101350000228F4D123E0FFF7D3FDC11B2D488142C1
:1013600017D8E0680007800F0328F4D117E0FFF7D3
:10137000C7FDC11B274881420BD8E0680007800FDA
:101380000128F4D10BE0FFF7BBFDC11B21488142CE
:1013900001D90320F8BDE0680007800FF3D11B4896
:1013A0000168C907C90FB1420DD901684908490050
:1013B00031430160006800E003E0C007C00FB042A5
:1013C00001D00120F8BD2878400706D5E068072144
:1013D00009028843E9680843E0602878000707D5D8
:1013E000E0680721C90288432969C9000843E06011
:1013F00000F036F8E168084A0906090F515CC84058
:10140000064908600020FFF771FEF8BD0020024089
:101410000010024088130000D02D000804000020B6
:10142000044805490068C968044A4905490F515CE8
:10143000C84070470400002000100240E92D000859
:10144000044805490068C968044A8904490F515C89
:10145000C84070470400002000100240E92D000839
:1014600010B5184AD1680C20084004280BD0082871
:1014700010D00C2810D050680004410F0120C00388
:10148000491C884010BD1068C00601D50E4810BD2B
:101490000E4810BD0E4810BD88020E4B000F185CA0
:1014A0000902D368890F491CDB0301D5084A05E00E
:1014B0001268D20601D5044A00E0044A5043FEF700
:1014C00019FE10BD0010024000093D000024F40088
:1014D00000127A00E02D0008FEB505007ED0FE4C1B
:1014E000E7680C20E66807400120000406402878E1
:1014F000C00747D0082F05D00C2F0AD101200004C7
:10150000864206D1206880033CD568680028E5D073
:1015100038E0012069680004814203D12168014359
:10152000216011E0052301221B04920499422168E5
:1015300002D111432160F1E781432160216801401C
:101540000091206890432060686800280DD0FFF764
:10155000D7FC009005E0FFF7D3FC0099401A6428FF
:101560007AD820688003F6D50CE0FFF7C9FC00901C
:1015700005E0FFF7C5FC0099401A6428F0D8206800
:101580008003F6D42878800755D50923E868042F0E
:101590000DD00C2F01D1002E09D000283BD021689E
:1015A000994301432160FFF7ABFC064627E0216821
:1015B000490701D5002891D061681F22120291438A
:1015C0002A69120211436160216899430143216035
:1015D000FFF746FFE16809060A0F00E079E1BF491D
:1015E000895CC840BE4908600020FFF77FFD0028E5
:1015F00072D120E0FFF784FC801B0228B0D820685D
:101600004007F7D560681F2109028843296909024C
:10161000084360600FE02068400840002060FFF74A
:101620006FFC064604E0FFF76BFC801B022897D88E
:1016300020684007F7D42878C0065FD5002F0CD06B
:10164000A869002849D02068FF21013108432060A3
:10165000FFF756FC06462DE0C0E02068800502D565
:10166000A8690028A7D06068072149038843296A30
:10167000084360606068297F0002000A0906084389
:101680006060286A410B0120C003491C8840E16862
:1016900009060A0F9149895CC840914908600020F9
:1016A000FFF724FD002817D128E0FFF729FC801B55
:1016B0000228A3D820688005F7D560680721490370
:1016C0008843296A084360606068297F0002000A35
:1016D00009060843606011E0E1E02168FF20013065
:1016E00081432160FFF70CFC064604E0FFF708FC8D
:1016F000801B022872D820688005F7D42878794E9C
:10170000000724D568690028306910D001210843FA
:101710003061FFF7F5FB009005E0FFF7F1FB009962
:10172000401A02285AD830698007F6D50FE04008E1
:1017300040003061FFF7E4FB009005E0FFF7E0FBBD
:101740000099401A022849D830698007F6D42878D1
:10175000400765D500200290A06BC00006D4A06BA6
:10176000012109070843A063012002905E48016837
:10177000C90511D40168821511430160FFF7C0FB50
:10178000009005E0FFF7BCFB0099401A642825D8BB
:1017900055480068C005F5D5FF20AA68013082428F
:1017A00003D131690143316111E001218902002A2D
:1017B00007D005231B029A4203D132690A433261E2
:1017C000EFE7326982433261306988433061A8684B
:1017D00000280FD0FFF794FB009007E05EE0FFF7D2
:1017E0008FFB0099411A4148814257D830698005E2
:1017F000F5D50DE0FFF784FB009006E0FFF780FBD6
:101800000099411A3948814248D830698005F5D499
:101810000298002804D0A06B012109078843A06327
:10182000686A002864D00C2F3ED0012636060228B4
:10183000206805D0B0432060FFF762FB05462FE02B
:10184000B0432060FFF75CFB074604E0FFF758FB5E
:10185000C01B022822D820688001F7D4E96AA86A50
:10186000E2680843296BFD231B049A431143084394
:10187000E060206830432060FFF742FB054604E04B
:10188000FFF73EFB401B022808D820688001F7D5EF
:101890002EE0FFF735FB401B022801D90320FEBDD7
:1018A00020688001F5D423E00128F8D0E068012108
:1018B0000904AA6A014091420BD10F218904EA6A06
:1018C0000140914205D1032189050840296B8842D6
:1018D0000ED00120FEBD000000100240D02D0008F7
:1018E00004000020401002400070004088130000F7
:1018F0000020EFE7094910B5401E884201D90120B8
:1019000010BD074C60610321081F00F0A9FA0020F8
:10191000A06107202061002010BD0000FFFFFF0034
:1019200000E000E0F0B502462032137E012B15D016
:10193000012717760223537605686C68AB6870261A
:10194000B4430E68496826438024A34319436E605C
:1019500000688160577600201076F0BD0220F0BD4F
:1019600070B5040005D025462035687E002802D0D9
:1019700006E0012070BD00202876204600F00AF81D
:1019800002206876211D206800F0F2FA01206876B6
:10199000002070BD00680449884204D10348816B6F
:1019A0001022114381637047001000400010024074
:1019B00070477047F8B502680446D06911689368AB
:1019C00005072D0F5BD0DD07ED0FFF2621360E40FA
:1019D0002E4367D0C60706D0CE0504D50126166271
:1019E000E26F3243E267870702220426002F06DAFD
:1019F000DF0704D027683A62E76F3743E767470796
:101A000006D5DB0704D023681E62E36F1343E36748
:101A1000020709D520220A402A4305D0236808225C
:101A20001A62E36F1343E367E26F002A2FD0800648
:101A300006D5880604D5216E002901D020468847A6
:101A4000E06F21688968490601D4000724D5204643
:101A500000F05AFB20688168490619D58168402248
:101A600091438160E06E002812D020498163E06ECE
:101A7000FFF74AF900280AD0E06E816B06E0850680
:101A800010D58D060ED5216E1CE020468847F8BD86
:101A90002046FFF78EFFF8BD2046FFF78AFF0020A3
:101AA000E067F8BDC50208D55B0206D50120000538
:101AB00010622046FFF77CFFF8BD030605D50B0634
:101AC00003D5616E0029E0D1F8BD4006FCD548067B
:101AD000FAD51368204640218B43136020216167AB
:101AE0000021616600F0D7F8F8BD0000F52000087D
:101AF00010B5040003D0606F002802D007E0012079
:101B000010BD002170200155204600F027F8242048
:101B1000606720680168490849000160204600F0BC
:101B200003FB0128ECD0606A002802D0204600F0B8
:101B30004BFA206841680922D20291434160206833
:101B400081682A2291438160206801680122114343
:101B50000160204600F09EFA10BD000010B586B06E
:101B6000044614216846FEF712FB15492068884296
:101B700024D11448416B0122920311434163C16A8D
:101B800001221143C162C06A6946104005900320DA
:101B90004002009002200190002002900320039058
:101BA0000420049005200007FFF7E2F80022114608
:101BB0001B20FFF7C9FA1B20FFF7BCFA06B010BDC7
:101BC0000038014000100240FFB50446406F83B06A
:101BD00017460D4620285CD1002D0AD0002F08D0D2
:101BE000A168C001814207D12069002804D1E8071B
:101BF00002D0012007B0F0BD204660300290007C8A
:101C0000012846D00298012101740020E0672120BC
:101C10006067FFF775F92646403601903782778274
:101C20000120A1680003814202D12069002802D06E
:101C30002F46002511E000270FE0002280212046DA
:101C400000F086FB002815D1002F15D021683878C8
:101C500088627F1C708A401E7082708A019B0028F7
:101C600006980090E9D100224021204600F070FB48
:101C7000002808D00320BDE728882168C005C00DD2
:101C80008862AD1CE6E72020606702990020087496
:101C9000B0E70220AEE77047FEE700001CB5002168
:101CA00018480091164A01910260C16301238363C1
:101CB00081601205036142600246C16020321370E8
:101CC000FF235170C23343628162117301638161EA
:101CD000042241634261C161FEF70AFF002801D07E
:101CE000FEF7BAFE08480090C00101906946054819
:101CF000FEF7B4FE002801D0FEF7AEFE1CBD0000CA
:101D0000002401400C00002020000014F0B587B032
:101D100014216846FEF73BFA1848C16A0125294399
:101D2000C162C16A29400591C26A02210A43C262A6
:101D3000C06A134C0840052636070590002221464C
:101D40003046FFF7D6F80F4F002270213846FFF7D4
:101D5000D0F800940024019502946946304603941B
:101D6000FFF706F8702000900294694601950394ED
:101D70003846FEF7FDFF07B0F0BD0000001002403E
:101D8000101800000004005010B5134811490160FC
:101D9000124941600021816001614161816101223C
:101DA000C161C2600162FFF7FBF8002801D0FEF7B5
:101DB00053FE00210848FFF7A9F8002801D0FEF7DC
:101DC0004BFE00210448FFF7C6F8002801D0FEF7BB
:101DD00043FE10BD00580040680000200E0900209E
:101DE0001CB500240E4800940C49019401600721A1
:101DF0008460416001214461C160FFF7B1FD0028AA
:101E000001D0FEF729FE0094694605480194FFF7CA
:101E100089FD002801D0FEF71FFE1CBD0010004008
:101E2000B400002010B50C480A490160E1214902C4
:101E3000416000218160C16001618161C1610C224A
:101E4000016242614162FFF753FE002801D0FEF7B4
:101E500003FE10BD00380140F00000207047000074
:101E60008307FF22DB0E9A408907090E994000285C
:101E70000BDA0007000F0838830808489B00181881
:101E8000C36993430B43C3617047830804489B00B5
:101E90001B181868904308431860704700ED00E075
:101EA00000E400E07047704710B5FFF703F910BD7C
:101EB00030B599B034216846FEF769F914210DA8B0
:101EC000FEF765F91C2112A8FEF761F912480168B6
:101ED0000322D2029143C2148918016002200090AB
:101EE0000024102009940125049003956846FFF70B
:101EF000F3FA0F200D9080200F900E951094002182
:101F000011940DA8FFF7D6F912A812951494FFF7B3
:101F10001FF919B030BD0000007000401048016882
:101F2000821511430160C1680E4A1140C160016809
:101F30000D4A1140016081684908490081600168CB
:101F40000122920491430160C168FD221204914371
:101F5000C160002101610549C0038860704700002D
:101F6000001002400C40FF88F6FFF6FE00ED00E096
:101F700070B5026801239B07114C124D984203D0A3
:101F8000A04201D0A84203D17026B2434E6832432A
:101F9000984203D0A04201D0A84204D103231B02DF
:101FA0009A43CB681A4380239A430B691A43026011
:101FB0008A68C262096881620121416170BD0000C6
:101FC000000801400014014010B5818CC90707D0FA
:101FD00001684A6801235B049A43836A1A434A6092
:101FE000818C890707D501684A6801231B049A433D
:101FF000C36A1A434A60818C490707D501684A6859
:1020000001239B049A43036B1A434A60818C09079E
:1020100007D501684A680123DB039A43436B1A43DF
:102020004A60818CC90607D50268916801231B03A9
:102030009943836B19439160818C890607D50168A8
:102040008A6801235B039A43C36B1A438A60818CBD
:10205000490612D503685A6801210905046C8A43B0
:1020600022435A60026C8A4207D1026851680323F6
:102070005B059943436C19435160818C090607D570
:1020800001684A680123DB04806C9A4302434A607A
:1020900010BD0000F8B500260446C667FEF730FF05
:1020A000054620680068124F000709D501212B461C
:1020B000002249052046009700F04AF900280DD17A
:1020C0002068006840070BD501212B4600228905B6
:1020D0002046009700F03CF9002801D00320F8BD0D
:1020E00020206067A067603426740020F8BD0000DF
:1020F000FFFFFF0110B5806A0022014640314A838C
:102100004A82FFF756FC10BD01680A68FF2321339D
:102110009A430A6001688A68520852008A60202146
:102120008167002101667047F8B504462669A268F8
:10213000E76932436669102000253E432368324335
:1021400078491E68784F3E4016431E6023685A68DF
:1021500003263603B243E66832435A602368A26915
:102160008B4201D0266A32439E680B273F02BE4352
:1021700016439E606D4E23686D4AB3420CD1D268FF
:102180009207920F06D0012A38D0022A34D0032AAF
:1021900020D11EE001201DE0664EB3420AD1D26874
:1021A0000C26324026D0042A28D0082A24D00C2A13
:1021B00010D10EE08B420DD1D66803229202164058
:1021C00018D001229202B61A18D0B61A14D096422C
:1021D00000D10820564A0126403A574FF6038B4259
:1021E00036D100280CD002280DD0042812D008289F
:1021F0001FD11CE00020EDE70220EBE70420E9E717
:10220000FFF70EF908E01068C00601D5384605E072
:102210004A4803E0FFF724F9002873D062685100B0
:102220005118814205D81103814202D303E03046A0
:10223000F4E7012566E0010E06025008002330187D
:102240005941FDF76DFF03210902411A3C4A55E04F
:10225000E169B14232D1030000F0DBF809070A0D51
:1022600006250606062B0600E3E7FFF7D9F81CE073
:10227000FFF7E6F819E010686168C00602D5480863
:10228000304A01E0304A48088018FDF733FF80B239
:1022900001462E4A10399142CBD8511C014000070B
:1022A000400F08432CE0FFF7DBF8616840004A0864
:1022B000EAE76168012248081204E5E7030000F03C
:1022C000A8F809070A0D06260606062C0600B0E740
:1022D000FFF7A6F81DE0FFF7B3F81AE01068616891
:1022E000C00602D54808C01902E014484A08101870
:1022F000FDF700FF80B20146144A1039914298D888
:102300002168C8600020206660662846F8BDFFF797
:10231000A7F861684A088018EAE7616848088019E8
:10232000E6E7000000480040F369FFEF0038014095
:10233000401002400044004000093D000024F40029
:10234000FFFC0F0000127A000048E801EFFF0000D8
:10235000FFB581B017460E4604460A9D09E0681C89
:1023600007D0FEF7CDFD0499401AA8420CD8002DE5
:102370000AD02068C1693046884318D00020B8428E
:10238000EDD0002005B0F0BD20680168FF22A13229
:1023900091430160206881684908490081602020DC
:1023A0006067A0670020603420740320EAE7012002
:1023B000E5E7000010B50248FFF7FCFA10BD000089
:1023C000F00000200FB410B503A9044B044A029892
:1023D00000F0F6F810BC08BC04B01847092D00083E
:1023E000080000202021020C01D010211046020A12
:1023F00001D010460839020901D01046091F820891
:1024000001D01046891E420801D0881E7047081A64
:10241000704730B47446641E2578641CAB4200D209
:102420001D46635D5B00E31830BC184702E008C836
:10243000121F08C1002AFAD170477047002001E03E
:1024400001C1121F002AFBD170470000F0B51FB474
:1024500086B00998089A030D0021024314D0514810
:10246000514A1818504305141198012810981AD091
:10247000281A401C00264D4F4D49009601910490AA
:10248000002812DA444211E01198012449A30128DE
:1024900001D11098C1430698119A84600360C2600C
:1024A00041600BB0F0BD4042E4E704462105002046
:1024B0003F4A001C51410391029012E0E00707D00F
:1024C00032463B4601990098FEF736F8019100909C
:1024D00032463B4610461946FEF72EF806460F4692
:1024E0006410002CEAD10498039B0028029A0999F1
:1024F000089806DAFEF720F8019B009AFEF71CF810
:1025000005E0FEF781F8019B009AFEF77DF804468E
:102510000E460022284BFEF70FF903D80020C043D7
:10252000014607E00022254B20463146FDF750FFCB
:10253000FEF7E2F8102409E0002C0ADB0A2200234F
:10254000FDF7EEFD079B30321A55641E02460A4322
:10255000F2D11122641C079B121B1C19119B012B29
:1025600003D0012308430ED10AE0084304D0112010
:1025700010900020119077E71098151A6D1E0BE04F
:102580001098824202DD00236D1C03E0824201DAD2
:1025900000236D1E002BEED0069811998260C16059
:1025A00030C07EE701FCFFFF104D0000000014402A
:1025B0000000F03F300000000000F0430000E03F6A
:1025C000FFB597B0064600251BE2252876D10024EA
:1025D0002746F749049400E00443761C3278012032
:1025E000203A90400842F7D130782A280ED00222B3
:1025F000307801463039092916D804990A235943FD
:10260000303940181443761C0490F1E7189802C83A
:1026100004911890002904DA012040030443484241
:10262000049002200443761C30782E2814D1042014
:1026300004437078761C2A2809D11898761C80C823
:10264000189009E00A214F43303FC719761C3078B3
:10265000014630390929F5D930786C2810D006DCCC
:102660004C281AD068280ED06A2817D104E07428A4
:1026700013D07A2812D110E00120400504430CE069
:102680000121090501E0032109050C43717881420C
:1026900003D1012000052418761C761C30786628AA
:1026A0000BD013DC58287DD009DC00287BD04528CE
:1026B000F6D04628F4D047281AD1A9E118E06328BB
:1026C00035D0642870D0652812D1A1E170286CD073
:1026D00008DC6728F1D069287DD06E280DD06F28DE
:1026E00006D1BCE073282ED0752873D0782859D035
:1026F0001A9A199990476D1C82E16002400F0228D6
:1027000009D003280DD00428189801680DD00D6059
:10271000001D189074E11898EA1701680D604A606E
:10272000F6E7189801680D80F2E70D70F0E7189849
:102730006A4601781172001D18900020507202A89C
:102740000090012005E0189802C818900020009120
:10275000C04361070ED5002101E00199491C019198
:10276000B94213DA8142F8DB019A0099895C0029A9
:10277000F3D10BE0002101E00199491C0191814254
:10278000FADB019A0099895C0029F5D10199049836
:102790001A9B471A21463846199A00F099FA4019AF
:1027A000019903E051E030E115E050E0451807E001
:1027B000009800990078491C00911A9A199990473D
:1027C0000198401E0190401CF2D1214638461A9BC8
:1027D000199A12E137E00A2000210090019160026D
:1027E000410F022907D0189A01CA1892C2179446BD
:1027F000032908D00AE01898C01DC108C90005C9FE
:102800001891944607E000B2C2179446042902D1F9
:1028100040B2C1178C4600226146944506DA0A464A
:102820000021404291418C462D2102E0210504D532
:102830002B216A461173012103E0E10701D0202119
:10284000F7E7029156E00A200AE0102008E0102085
:1028500000900021042004430191082703E0082090
:102860000021019100906002410F022907D0189ABF
:1028700001CA189200229446032908D008E018984B
:10288000C01DC108C90005C91891944603E080B273
:10289000042900D1C0B20021029121072AD5317844
:1028A0000D91702906D0009A1021019B4A401A43CD
:1028B00005D00EE040216A461173012108E061460F
:1028C000014306D030216A4611730D9951730221DC
:1028D0000291009A0821019B4A401A430AD161469D
:1028E000014301D1610705D530216A4611730121E9
:1028F0007F1E02913178582904D02EA10E910DA986
:102900000D910DE030A1F9E76146019B009AFDF7BA
:1029100007FC0E9B8C469B5C0D9A521E0D92137009
:1029200061460143F0D10D9805A9081A20300190A5
:10293000600703D501200004844300E001270198CB
:10294000874201DD381A00E000200199009041180B
:10295000029809180498401A0490E00306D421460E
:102960001A9B199A049800F0B3F94519002706E05C
:1029700003A81A9AC05D199990476D1C7F1C029894
:102980008742F5DBE0030CD521461A9B199A04987F
:1029900000F09EF9451904E01A9A302019999047E1
:1029A0006D1C0099481E00900029F5DC1FE0000016
:1029B0000928010030313233343536373839616215
:1029C00063646566000000003031323334353637D9
:1029D0003839414243444546000000000D980D99A6
:1029E0000078491C0D911A9A199990476D1C01990C
:1029F000481E01900029F1DC4DE100F059F945191C
:102A0000761C3078002800D0DFE528461BB0F0BDEA
:102A1000600700D406271898C01DC108C90048687F
:102A20000A680831C30FDB071891190001D09CA177
:102A300008E0210501D59BA104E0E10701D09AA19E
:102A400000E09AA14300109130785B0865280CD013
:102A500006DC452809D046281DD0472841D141E051
:102A6000662818D067283CD13CE00021112F01DBFB
:102A7000112000E0781C0191009008A911A8FFF72F
:102A8000E5FC139905910021119A15927F1C12986B
:102A90000197009150E00120C007039001200190B0
:102AA00008A9009711A8FFF7D1FC139A1499059271
:102AB0000022119B009212981593059A0192002909
:102AC00001D0104602E0791C40180190381A01D557
:102AD000019804E04042401E0090781C0190C01B09
:102AE000029043E0012F00DA01270021112F01DDC0
:102AF000112000E038460191009008A911A8FFF7C5
:102B0000A5FC13990591119A002112981592009134
:102B1000019721070CD40599B94201DB019900E026
:102B20000191012904DD159A491E515C302906D016
:102B3000B84201DA011D05DA0121029115E001997F
:102B4000491EEDE7002805DC009941180091019924
:102B5000091A03E0019A411C914200DD019100999C
:102B6000401A401C02900120C0070390200706D4A1
:102B700002990198814202DB0020C04302900020AC
:102B80006946C87707AF012103980337C907884210
:102B900024D0022011902B201290039800280CDAE8
:102BA000404203902D20129007E00A210398FDF780
:102BB000A1FA30317F1E039039701199481E11908F
:102BC0000029F2DC03980028EFD1791E12980870D2
:102BD0003078202108404530BF1E387006A8C01B41
:102BE000C01D039010980078002800D001200199A2
:102BF00041180298C0170918039809180498401A38
:102C0000401E0490E00306D421461A9B199A0498AA
:102C100000F05EF8451910980078002803D01A9A41
:102C2000199990476D1CE00324D521461A9B199AE7
:102C3000049800F04DF845191CE00098002807DBC7
:102C400000990598884203DD1598405C199901E0C8
:102C5000199930201A9A904700986D1C401C0090DA
:102C60000298401E0290002804D11A9A2E20199929
:102C700090476D1C0199481E01900029DDDC05E09C
:102C800038781A9A7F1C199990476D1C0399481E31
:102C900003900029F4DC21461A9B199A0498ACE6AB
:102CA0002D0000002B0000002000000000000000AC
:102CB000F8B5044600251E461746880404D405E0EE
:102CC00039462020B0476D1C641EF9D52846F8BD52
:102CD000FFB50446002581B01E46C80301D5302744
:102CE00000E02027880404D505E038460399B04762
:102CF0006D1C641EF9D5284605B0F0BD4100401892
:102D0000401EFDD27047000001B5044B0122694608
:102D10000348FEF759FF009808BD0000FFFF0000C0
:102D2000F0000020FEF7CEF9FFF7C2F800252C4690
:102D3000FEF7ECFFFFF728F8FFF774F8FFF750F8FD
:102D4000FEF7ACFFFF26F53605E017A0FFF73AFBCC
:102D50003046FDF7FFFFFDF7F3FD0028F5D1FDF745
:102D6000C1FD19204001FDF7F5FF154E154F0A343E
:102D700004E000246D1C3C2D00D10025FDF7B2FDC0
:102D8000FDF78BFA3146FDF74AFAFDF7AAFA02463B
:102D90000B460DA0FFF716FB3846FDF7DBFF0A34A4
:102DA0003C2CE8D1E5E70000445331384232302072
:102DB000436865636B204661696C6564210D0A0098
:102DC0000000204110270000313A25332E316600E3
:102DD00000000000000000000102030406070809CB
:102DE000030406080C101820300000000001020344
:102DF00004000000142E0008000000200C00000059
:102E00002C240008202E00080C000020640500007F
:102E10003C2400080000000000002000000000002A
:04000005080000C12E
:00000001FF
